:100000000C9466010C948E010C948E010C948E015C
:100010000C948E010C948E010C948E010C948E0124
:100020000C948E010C948E010C948E010C948E0114
:100030000C948E010C948E010C948E010C948E0104
:100040000C9421240C948E010C9447280C94952830
:100050000C948E010C948E010C948E010C948E01E4
:100060000C948E010C948E013C76657273696F6EF0
:1000700020302E3934343E00467265652052414DA1
:100080003A20004552524F523A200053797320765D
:100090006F6C74733A200053797320766F6C7473AD
:1000A000206368617267696E673A20005379732034
:1000B000766F6C74732069646C653A2000626174B9
:1000C00074506C757350696E204F4E006261747489
:1000D000506C757350696E204F464600637572729E
:1000E000656E745A65726F4F66667365743A005335
:1000F000616D706C652073697A653A20003E00205E
:1001000000200020002000200020002000200020EF
:10011000003C0041444A555354494E472000616415
:100120006A416D70735F4F4E200061646A566F6C58
:1001300074735F4F4E200063656C6C5368756E740A
:10014000335F4F4E200063656C6C5368756E74327C
:100150005F4F4E200063656C6C5368756E74315F41
:100160004F4E200074617267657420416D70733A60
:10017000200074617267657420566F6C74733A2046
:100180000070777250574D3A200049444C45205436
:100190004F54414C20566F6C74733A200049444CC4
:1001A0004520566F6C747320333A200049444C4507
:1001B00020566F6C747320323A200049444C45201D
:1001C000566F6C747320313A2000434841524749BE
:1001D0004E4720544F54414C20566F6C74733A2054
:1001E000004348415247494E4720566F6C74732074
:1001F000333A20004348415247494E4720566F6CDE
:10020000747320323A20004348415247494E4720F8
:10021000566F6C747320313A20004348415247496D
:100220004E472063757272656E7420414D50533A8B
:100230002000544F54414C20766F6C74733A200068
:10024000766F6C747320333A2000766F6C74732071
:10025000323A2000766F6C747320313A2000437577
:100260007272656E7420416D70733A200000000058
:1002700000240027002A0000000000250028002B91
:1002800000000000002300260029000404040404E8
:100290000404040202020202020303030303030133
:1002A000020408102040800102040810200102040A
:1002B00008102000000007000201000003040600EF
:1002C00000000000000000009F02012A11241FBE50
:1002D000CFEFD8E0DEBFCDBF15E0A0E0B1E0ECECA1
:1002E000F9E502C005900D92A430B107D9F716E0E8
:1002F000A4E0B5E001C01D92A739B107E1F712E013
:10030000CCECD2E004C02297FE010E94E02CC83C55
:10031000D107C9F70E9430280C94E42C0C940000FB
:10032000EF92FF920F931F937A018B01AA2797FDFB
:10033000A095BA2FBC01CD010E945B2BA8019701AB
:100340000E940F2C20E030EC4FE754E40E94C02ABA
:1003500020E030E040E250E40E94572A24EA30E7EF
:100360004DE35EE30E94C02A1F910F91FF90EF9032
:1003700008956F927F928F929F92AF92BF92CF9289
:10038000DF92EF92FF920F931F933A014B0181305E
:10039000910599F4222389F0A0906B05B0906C052B
:1003A000C0906D05D0906E0520916F05309170055D
:1003B000409171055091720515C082309105D9F4B4
:1003C0002223C9F0A0906F05B0907005C090710510
:1003D000D090720520916B0530916C0540916D05B0
:1003E00050916E05E0907305F090740500917505CD
:1003F000109176056EC083309105D9F42223C9F09F
:10040000A0907305B0907405C0907505D0907605E6
:1004100020916B0530916C0540916D0550916E05F2
:10042000E0906F05F09070050091710510917205D4
:1004300050C08130910599F4222389F4A0907B0566
:10044000B0907C05C0907D05D0907E0520917F0501
:1004500030918005409181055091820515C0823010
:100460009105D9F42223C9F4A0907F05B0908005AE
:10047000C0908105D090820520917B0530917C054C
:1004800040917D0550917E05E0908305F0908405B4
:1004900000918505109186051CC00397D1F4222395
:1004A000C1F4A0908305B0908405C0908505D090DC
:1004B000860520917B0530917C0540917D0550910A
:1004C0007E05E0907F05F0908005009181051091F8
:1004D0008205C601B5010E94572AA40193010E941A
:1004E0000B2C1816ECF0C601B501A80197010E946B
:1004F000572AA40193010E940B2C181614F010E047
:1005000010C010E0C601B5012091ED043091EE0459
:100510004091EF045091F0040E940B2C18160CF43B
:1005200011E0812F1F910F91FF90EF90DF90CF90FE
:10053000BF90AF909F908F907F906F900895609143
:10054000C6047091C7048091C8049091C9042DEC31
:100550003CEC4CE45DE30E94572A609336057093AF
:10056000370580933805909339056091E7047091C1
:10057000E8048091E9049091EA042AE939E949E123
:100580005FE30E94572A6093AD057093AE05809398
:10059000AF059093B005089581E796E068E670E0B6
:1005A0000E940B260895DF92EF92FF920F931F9304
:1005B000482FD92E8B018FEDE82E85E0F82EC7014C
:1005C0000E9490230F5F1F4FC701B8014D2D0E945D
:1005D00090231F910F91FF90EF90DF90089560910D
:1005E0005B0570915C0580915D0590915E052091A1
:1005F0005F053091600540916105509162050E9450
:10060000582A209163053091640540916505509109
:1006100066050E94582A9B01AC01609167057091A4
:1006200068058091690590916A050E940B2C181647
:1006300024F58091EB049091EC04019731F18091C5
:100640009E0590919F05823091058CF010929F0538
:1006500010929E0581E090E09093EC048093EB046F
:1006600081E796E060E071E00E941D280895019600
:1006700090939F0580939E05089510929F05109278
:100680009E051092EC041092EB040895EF92FF92F5
:100690000F931F939C018130910539F182309105B0
:1006A0001CF4009749F0FFC082309105B9F1833006
:1006B000910509F0F8C085C08091CB059091CC05DB
:1006C000892B09F4F0C08091900590919105892BB8
:1006D00009F0E9C01092CC051092CB051092CA0522
:1006E0001092C9058DE060E0DCC08091CB0590914F
:1006F000CC05019709F4D7C08091900590919105A0
:10070000892B09F0D0C03093CC052093CB053093D2
:10071000CA052093C9058DE061E0C3C02091C505DD
:100720003091C6054091C7055091C8052115310586
:100730004105510531F08091CB059091CC05029790
:1007400079F082E090E09093CC058093CB0581E036
:1007500090E09093CA058093C9058DE061E022C0C6
:100760008091040590910505A0910605B0910705BB
:1007700082179307A407B50708F495C08091C905AF
:100780009091CA05019729F41092CA051092C905E3
:1007900006C081E090E09093CA058093C9058DE082
:1007A0006091C9050E944A25809104059091050534
:1007B000A0910605B0910705845D9E4FAF4FBF4FD6
:1007C00036C08091900590919105892B09F06BC0FE
:1007D000E090C505F090C6050091C7051091C805C9
:1007E000E114F1040105110531F08091CB059091E0
:1007F000CC05039729F183E090E09093CC0580939A
:10080000CB0581E090E09093CA058093C9058DE007
:1008100061E00E944A258091040590910505A09110
:100820000605B09107058A5B9F4FAF4FBF4F80937E
:10083000C5059093C605A093C705B093C80533C0FE
:10084000209104053091050540910605509107055A
:100850002E153F054007510730F18091C905909151
:10086000CA05019749F41092CA051092C90524528D
:100870003A4F4F4F5F4F0AC081E090E09093CA0516
:100880008093C9052A5B3F4F4F4F5F4F2093C505AB
:100890003093C6054093C7055093C8058DE060911D
:1008A000C9050E944A251F910F91FF90EF9008956E
:1008B00082E061E00E944A251092F10480918F0548
:1008C000882331F081E796E06CE071E00E941D28FA
:1008D000089582E060E00E944A258091F104882317
:1008E00051F480918F05882331F081E796E064E22E
:1008F00071E00E941D2881E08093F104089583E057
:1009000061E00E944A2580918F05882331F081E7BC
:1009100096E06EE371E00E941D28089581309105F4
:1009200089F4662341F088E061E00E944A2581E075
:1009300080934605089588E060E00E944A25109261
:10094000460508958230910589F4662341F087E0D9
:1009500060E00E944A2581E080934705089587E082
:1009600061E00E944A25109247050895039781F49B
:10097000662341F084E060E00E944A2581E0809394
:100980004805089584E061E00E944A2510924805D8
:1009900008958DE061E00E944A2560E07DE780E0F7
:1009A00090E00E9477248DE060E00E944A2560E09C
:1009B0007DE780E090E00E9477248DE061E00E9476
:1009C0004A2560E07DE780E090E00E9477248DE09A
:1009D00060E00E944A2560E07DE780E090E00E94B0
:1009E00077248DE061E00E944A2560E07DE780E0A9
:1009F00090E00E9477248DE060E00E944A2560E04C
:100A00007DE780E090E00E9477240895DF92EF92E6
:100A1000FF920F931F938C019FEDE92E95E0F92E25
:100A2000C701B8010E948923D82E0F5F1F4FC7014D
:100A3000B8010E9489236D2D0E943F281F910F91BC
:100A4000FF90EF90DF900895FF920F931F93CF9345
:100A5000DF9381E796E064E571E00E9420278091B2
:100A6000DB049091DC04089721F0FF24C8E0D0E07B
:100A70001BC081E796E062E671E039C0CE010E94BA
:100A800006058C01FF2031F081E796E065E671E014
:100A90000E94202781E796E0B8014AE050E00E94DA
:100AA000EE262296FF24F3948091DB049091DC04DF
:100AB0000197C817D90714F380919005909191057B
:100AC0000817190781F081E796E065E671E00E945A
:100AD0002027609190057091910581E796E04AE0AA
:100AE00050E00E94EE2681E796E067E671E00E9402
:100AF0001D28DF91CF911F910F91FF9008951092C3
:100B0000200510921F0585E060E070E00E94C1237F
:100B100010921D0510921C0510921E0585E090E0B4
:100B20009093B9048093B80408950E947F0581E0F2
:100B300090E060E00E948E0482E090E060E00E941D
:100B40008E0483E090E060E00E948E0408950E948D
:100B5000950510922D0580E090E00E9446030895CF
:100B60002F923F924F925F926F927F928F929F92BD
:100B7000AF92BF92CF92DF92EF92FF920F931F93AB
:100B8000CF93DF93EC010F2EF3E32F2EF3E33F2EF1
:100B9000F3E74F2EF0E45F2EF02D0F2EF0E06F2ED6
:100BA000F0E07F2EF0E68F2EF0E49F2EF02D0F2E3A
:100BB000FDECAF2EFCECBF2EFCE5CF2EF0E4DF2EDB
:100BC000F02D0F2EF0E0EF2EF0E0FF2EF0E00F2FD3
:100BD000FFE31F2FF02D8091900590919105C8178C
:100BE000D90761F1209751F16091DB047091DC0429
:100BF000CE010E94D3026091DB047091DC046E5F31
:100C00007F4F80E090E00E94D3028091DB049091BE
:100C1000DC0402969093DC048093DB0480918F05C2
:100C2000882331F081E796E069E671E00E941D2893
:100C3000D0939105C09390050E942405D09391050F
:100C4000C093900582E090E00E94460320919005B9
:100C5000309191052115310529F480E090E00E9442
:100C6000460348C0243131050CF444C0C9014497FF
:100C7000449740F0C90188974497C0F1C901CC97C7
:100C8000449778F50E94A70586E696E6A6E7B0E4C5
:100C90008093C6049093C704A093C804B093C9047A
:100CA000209236053092370540923805509239052A
:100CB0006092D6047092D7048092D8049092D9049E
:100CC000A092ED04B092EE04C092EF04D092F00432
:100CD000E092CA04F092CB040093CC041093CD04AC
:100CE00009C0205530402431310520F41092DA0437
:100CF0000E94A7058091DB049091DC044897F4F0F2
:100D00000E94B1068823D1F4A8E0B0E0B093DC04DF
:100D1000A093DB04809190059091910568E070E0CC
:100D20000E94D3028091DB049091DC0402969093A0
:100D3000DC048093DB04CEE3D0E04DCFDF91CF9194
:100D40001F910F91FF90EF90DF90CF90BF90AF90E9
:100D50009F908F907F906F905F904F903F902F90DB
:100D60000895CF93DF93C8E0D0E008C0CE010E9481
:100D70000605889714F080E025C022968091DB0458
:100D80009091DC048C179D078CF7C8E0D0E007C079
:100D90008FED95E0BE0140E00E9490232196809166
:100DA000DB049091DC0401968C179D078CF788E09A
:100DB00090E09093DC048093DB0480E090E00E945C
:100DC000B00581E0DF91CF91089560915705709152
:100DD00058058091590590915A052091CA04309187
:100DE000CB044091CC045091CD040E94572A29E2B3
:100DF0003CE54FE05EE30E940B2C181694F48091C2
:100E0000BB059091BC05853191052CF083E590E000
:100E10000E94B00506C001969093BC058093BB0567
:100E200008951092BC051092BB0508956091570576
:100E3000709158058091590590915A0520E030E055
:100E400040E05FE30E94BC2A8823CCF480911F0518
:100E500090912005843B910591F48091B905909182
:100E6000BA05893291052CF08AE290E00E94B00523
:100E700006C001969093BA058093B9050895109223
:100E8000BA051092B90508956091570570915805FB
:100E90008091590590915A052AE939E949E95EE3BB
:100EA0000E940B2C1816D4F480911F0590912005F8
:100EB000892BA1F48091B3059091B40585309105FB
:100EC0003CF082E590E00E94B0050E94690406C0F3
:100ED00001969093B4058093B30508951092B405DC
:100EE0001092B305089583E060E00E944A25809146
:100EF0008F05882331F081E796E061E871E00E9478
:100F00001D288091E5049091E604019751F060E07E
:100F100072EE84E090E00E9477248DE390E00E94DE
:100F2000B005089560915705709158058091590555
:100F300090915A0520E030E040E750EC0E94BC2A36
:100F40008823BCF48091A7059091A8058330910572
:100F50005CF081E796E068E971E00E941D2810923C
:100F6000A8051092A70505C001969093A805809347
:100F7000A70560915705709158058091590590918A
:100F80005A0520E030E048E850EC0E94BC2A882353
:100F9000BCF48091A9059091AA05833091055CF07D
:100FA00082E090E00E94B0050E9473071092AA05AB
:100FB0001092A905089501969093AA058093A9051A
:100FC0000895AF92BF92CF92DF92EF92FF920F936C
:100FD0001F931092C1051092C2051092C305109282
:100FE000C4058091F1048823D9F080911F05909168
:100FF000200518161906A4F0609167057091680520
:101000008091690590916A052091AD053091AE05FA
:101010004091AF055091B0050E94BC2A88231CF472
:1010200081E090E04DC0A090BD05B090BE05C0909D
:10103000BF05D090C005609157057091580580910B
:10104000590590915A05A60195010E94572A9B01C6
:10105000AC0168E17AEF88E29BEB0E94572A7B01A2
:101060008C016093BD057093BE058093BF0590937E
:10107000C00520E030E040E050E00E940B2C181644
:101080005CF4C801B70120E030E040E85EE30E9474
:101090000B2C18165CF017C0C801B70120E030E037
:1010A00040E85EEB0E94BC2A88236CF4A092BD0548
:1010B000B092BE05C092BF05D092C00581E590E018
:1010C0000E94B00548C080918F05882341F181E7D7
:1010D00096E067EA71E00E941D28C601B5012091E3
:1010E000BD053091BE054091BF055091C0050E94DD
:1010F000BC2A8823A1F081E796E066EB71E00E94AC
:1011000020274091BD055091BE056091BF057091AB
:10111000C00581E796E022E030E00E940A28609155
:10112000BD057091BE058091BF059091C00520E07E
:1011300030E04AE754E40E940F2C20E030E04AE718
:1011400054E40E94582A0E94282BDC01CB0164E061
:1011500070E00E94D3021F910F91FF90EF90DF90FB
:10116000CF90BF90AF9008958091E5049091E604F0
:10117000019791F560916705709168058091690507
:1011800090916A052091AD053091AE054091AF0573
:101190005091B0050E94BC2A8823F4F48091B105D7
:1011A0009091B2058A3091058CF01092B2051092A0
:1011B000B10581E796E068EC71E00E941D280E946D
:1011C000A70584E090E00E94B005089501969093F1
:1011D000B2058093B10508951092B2051092B10541
:1011E000089560915B0570915C0580915D0590911B
:1011F0005E0520915F053091600540916105509139
:1012000062050E94582A2DEC3CEC4CE45EE30E94FF
:10121000BC2A88233CF483E090E00E94B0050E9441
:10122000A70508958091900590919105039721F469
:1012300080E090E00E94B00508958091A605882383
:10124000F9F40E94A70581E796E061ED71E00E9444
:101250001D288091040590910505A0910605B09187
:1012600007058053984FAF4FBF4F8093A0059093D1
:10127000A105A093A205B093A30581E08093A605E4
:101280000895EF92FF920F931F938091E504909140
:10129000E604892B09F0F9C0E090ED04F090EE042B
:1012A0000091EF041091F00460915B0570915C0572
:1012B00080915D0590915E05A80197010E94BC2A6E
:1012C00087FD1CC060915F0570916005809161058C
:1012D00090916205A80197010E94BC2A87FD0EC06B
:1012E0006091630570916405809165059091660534
:1012F000A80197010E94BC2A88239CF58091A4052F
:101300009091A5058035910534F11092A5051092B4
:10131000A4050E941D096091ED047091EE04809176
:10132000EF049091F0042DEC3CEC4CE450E40E946E
:10133000BC2A8823D1F486E090E00E94B005809119
:101340008F05882309F4A1C081E796E06CED71E078
:101350000E941D289AC001969093A5058093A4052C
:1013600004C01092A5051092A40560915B057091D0
:101370005C0580915D0590915E0520E030E040E6DF
:1013800050E40E94BC2A87FD21C060915F057091E6
:101390006005809161059091620520E030E040E6B3
:1013A00050E40E94BC2A87FD11C0609163057091D2
:1013B0006405809165059091660520E030E040E687
:1013C00050E40E94BC2A88230CF05BC08091AB05DE
:1013D0009091AC05803591050CF44DC01092AC0590
:1013E0001092AB058091CB059091CC050397F1F15C
:1013F0006091DD047091DE048091DF049091E0043F
:101400002091920530919305409194055091950556
:101410000E94572A23E333E343E75FE30E94C02A95
:101420006093DD047093DE048093DF049093E00406
:101430000E94282BDC01CB0162E070E00E94D30205
:101440006091DD047091DE048091DF049091E004EE
:101450002DEC3CEC4CE45DE30E940F2C6093920574
:1014600070939305809394059093950583E090E0A5
:101470000E9446030AC001969093AC058093AB0589
:1014800004C01092AC051092AB051F910F91FF9014
:10149000EF900895EF92FF920F931F9360915B0579
:1014A00070915C0580915D0590915E0520915F05CE
:1014B0003091600540916105509162050E94582A63
:1014C0002091630530916405409165055091660552
:1014D0000E94582A7B018C016091D6047091D70438
:1014E0008091D8049091D90420E030E040E450E4A9
:1014F0000E940F2C9B01AC01C801B7010E94BC2ABD
:101500008823ACF46091C6047091C7048091C8042C
:101510009091C9042DEC3CEC44E850E40E94BC2AB4
:10152000882329F48DE290E00E94B00528C00E9433
:10153000A7056091C6047091C7048091C80490917A
:10154000C9042DEC3CEC44E850E40E94BC2A8823FA
:10155000B1F48091DD049091DE04A091DF04B0919C
:10156000E0048093920590939305A0939405B09323
:10157000950581E796E061EF71E00E941D281F91BB
:101580000F91FF90EF900895EF92FF920F931F93AA
:101590007B018C018091900590919105039749F111
:1015A00081E080932D050E9495058091040590911E
:1015B0000505A0910605B09107058E0D9F1DA01F82
:1015C000B11F8C53964FAF4FBF4F80932E05909312
:1015D0002F05A0933005B0933105845C9940A0405D
:1015E000B04080933A0590933B05A0933C05B0939F
:1015F0003D051F910F91FF90EF900895EF92FF929C
:101600000F931F93E0906705F090680500916905BE
:1016100010916A05C801B7012091E7043091E804F0
:101620004091E9045091EA040E940B2C88230CF4A9
:1016300088C010929B0510929A058091E5049091C4
:10164000E604019709F4EAC080919C0590919D05FC
:10165000823091050CF46FC010929D0510929C058C
:1016600081E090E09093E6048093E50481E796E0C2
:101670006BEF71E00E941D288091DA04882309F441
:10168000CDC0E0903605F0903705009138051091F7
:10169000390560915B0570915C0580915D059091C5
:1016A0005E05A80197010E940B2C8823FCF0609135
:1016B0005F05709160058091610590916205A801B8
:1016C00097010E940B2C88238CF060916305709128
:1016D00064058091650590916605A80197010E94B7
:1016E0000B2C88231CF00E944A0A98C080918F0519
:1016F000882331F081E796E064E072E00E941D28C3
:1017000060E177E280E090E00E94C40A80910405E5
:1017100090910505A0910605B091070588579C4E4C
:10172000AF4FBF4F8093C1059093C205A093C305EF
:10173000B093C40573C0019690939D0580939C055A
:101740006DC010929D0510929C0560915B05709193
:101750005C0580915D0590915E0520915F0530915B
:10176000600540916105509162050E94582A2091C0
:1017700063053091640540916505509166050E94AE
:10178000582A9B01AC01C801B7010E94BC2A181657
:101790000CF440C010929D0510929C058091E504C8
:1017A0009091E604892BD1F180919A0590919B0547
:1017B000823091054CF110929B0510929A0510927F
:1017C000E6041092E50481E796E063E172E00E948E
:1017D0001D280E9458041092C1051092C205109253
:1017E000C3051092C4058091DA048823B9F0809172
:1017F0008F05882331F081E796E06EE172E00E9468
:101800001D280E94A7050AC0019690939B0580930E
:101810009A0504C010929B0510929A051F910F9192
:10182000FF90EF9008952F923F924F925F926F92A8
:101830007F928F929F92AF92BF92CF92DF92EF9260
:10184000FF920F931F93DF93CF9300D000D0CDB7BB
:10185000DEB78091040590910505A0910605B09131
:10186000070589839A83AB83BC8380931805909383
:101870001905A0931A05B0931B0580911C058823B8
:10188000D9F06090B0047090B1048090B204909050
:10189000B304A0904205B0904305C0904405D09099
:1018A00045050F2EFAE02F2EF7ED3F2EF3EA4F2ECF
:1018B000FCE35F2EF02D1AC06090B4047090B50464
:1018C0008090B6049090B704A0908B05B0908C05E2
:1018D000C0908D05D0908E050F2EF9E22F2EFCE5DD
:1018E0003F2EFFE84F2EFDE35F2EF02DC601B50120
:1018F000A40193010E94572A7B018C0120E030E073
:1019000040E050E00E940B2C181624F017FB1095B5
:1019100017F91095C801B701A20191010E940B2C83
:1019200088230CF4F7C080911E05882309F04AC073
:1019300081E080931E0589819A81AB81BC8180936F
:10194000230590932405A0932505B0932605C60191
:10195000B501A40193010E94BC2A88231CF481E0F4
:1019600090E002C08FEF9FEF9093220580932105B6
:10197000C201B10120E030E040E850E40E940F2CA9
:101980009B01AC01C801B7010E940B2C18161CF476
:1019900085E090E002C081E090E09093B9048093EC
:1019A000B80420912105309122058091B8049091CE
:1019B000B904D901A89F9001A99F300DB89F300D9F
:1019C00011244EC0C601B501A40193010E94BC2A96
:1019D0008823BCF480912105909122058F5F9F4F51
:1019E00081F481E090E09093B9048093B8049093DF
:1019F00022058093210580911F0590912005019675
:101A000035C0C601B501A40193010E940B2C181624
:101A1000BCF480912105909122058130910581F4DB
:101A20009093B9048093B8048FEF9FEF90932205B1
:101A30008093210580911F0590912005019716C084
:101A400020912105309122058091B8049091B9042C
:101A5000F901E89F9001E99F300DF89F300D1124A6
:101A600080911F0590912005820F931F9093200570
:101A700080931F0580911F0590912005853B91055E
:101A80003CF084EB90E09093200580931F0506C006
:101A900097FF04C01092200510921F0560911F054A
:101AA0007091200585E00E94C123209104053091AA
:101AB000050540910605509107058091BE0490915F
:101AC000BF04A091C004B091C104820F931FA41F52
:101AD000B51F80930C0590930D05A0930E05B09350
:101AE0000F0580ED97E0A0E0B0E08093BA049093FA
:101AF000BB04A093BC04B093BD0428533F4F4F4F89
:101B00005F4F209327053093280540932905509374
:101B10002A0502C010921E050F900F900F900F9093
:101B2000CF91DF911F910F91FF90EF90DF90CF90B9
:101B3000BF90AF909F908F907F906F905F904F90ED
:101B40003F902F90089560911F057091200585E0CA
:101B50000E94C1232091040530910505409106059E
:101B6000509107058091BE049091BF04A091C004DC
:101B7000B091C104820F931FA41FB51F80930C0561
:101B800090930D05A0930E05B0930F0580ED97E09F
:101B9000A0E0B0E08093BA049093BB04A093BC048F
:101BA000B093BD0428533F4F4F4F5F4F20932705FD
:101BB000309328054093290550932A0510921E055D
:101BC00008958F929F92AF92BF92CF92DF92EF9241
:101BD000FF920F931F93E0900405F090050500918C
:101BE0000605109107058091C2049091C304A0914D
:101BF000C404B091C504A8019701281B390B4A0BF6
:101C00005B0B8091320590913305A0913405B09122
:101C1000350582179307A407B50708F0F1C0E092D5
:101C20003205F0923305009334051093350584ECAA
:101C300099E0A0E0B0E08093C2049093C304A09325
:101C4000C404B093C504A0904605909047058090C9
:101C5000480581E090E04DEC5CEC6CE47DE321E034
:101C60000E94B901B82E882311F0BB24B39482E0FE
:101C700090E04DEC5CEC6CE47DE321E00E94B90166
:101C8000C82E882311F0CC24C39483E090E04DEC5F
:101C90005CEC6CE47DE321E00E94B901D82E88233E
:101CA00011F0DD24D394BB2041F1E0906B05F0905E
:101CB0006C0500916D0510916E05C801B70120916A
:101CC0006F053091700540917105509172050E9429
:101CD000BC2A882374F4C801B701209173053091A0
:101CE000740540917505509176050E94BC2A87FDC8
:101CF00004C081E090E061E003C081E090E060E03A
:101D00000E948E04CC2041F1E0906F05F0907005A8
:101D10000091710510917205C801B70120916B0502
:101D200030916C0540916D0550916E050E94BC2A62
:101D3000882374F4C801B7012091730530917405AC
:101D400040917505509176050E94BC2A87FD04C01C
:101D500082E090E061E003C082E090E060E00E94F9
:101D60008E04DD2041F1E0907305F0907405009140
:101D7000750510917605C801B70120916B0530916A
:101D80006C0540916D0550916E050E94BC2A882318
:101D900074F4C801B70120916F053091700540912E
:101DA0007105509172050E94BC2A87FD04C083E032
:101DB00090E061E003C083E090E060E00E948E0468
:101DC000BB2021F4CC2011F4DD2061F080E29EE400
:101DD000A0E0B0E08093C2049093C304A093C40435
:101DE000B093C504809146058A1541F4809147055A
:101DF000891521F480914805881511F00E94A30DE2
:101E00001F910F91FF90EF90DF90CF90BF90AF9018
:101E10009F908F900895EF92FF920F931F93E09001
:101E20000405F09005050091060510910705E09264
:101E30002E05F0922F050093300510933105809107
:101E40003A0590913B05A0913C05B0913D05A80154
:101E50009701281B390B4A0B5B0B8091CE049091A4
:101E6000CF04A091D004B091D10482179307A407A6
:101E7000B50778F480918F05882331F081E796E0EB
:101E80006EE272E00E941D280E94A7058EE290E09B
:101E90003BC08091900590919105039719F40E94A1
:101EA000A70566C160916B0570916C0580916D0509
:101EB00090916E0524EA30E745E850E40E940B2C2F
:101EC000181604F160916F0570917005809171058D
:101ED0009091720524EA30E745E850E40E940B2C0B
:101EE000181684F0609173057091740580917505E2
:101EF0009091760524EA30E745E850E40E940B2CE7
:101F000018162CF48BE290E00E94B00531C160916C
:101F10008B0570918C0580918D0590918E052DEC2F
:101F20003CEC4CE45EE30E94BC2A882304F58091DB
:101F30001C058823E1F080913E0590913F05A0911A
:101F40004005B0914105E81AF90A0A0B1B0B809174
:101F5000D2049091D304A091D404B091D5048E15ED
:101F60009F05A007B10758F40E944A0A01C1E092F8
:101F70003E05F0923F05009340051093410581E036
:101F800090E00E944603E090CA04F090CB040091D8
:101F9000CC041091CD0460916B0570916C0580911B
:101FA0006D0590916E052DEC3CEC4CE450E40E94E4
:101FB000BC2A87FD20C060916F05709170058091EB
:101FC0007105909172052DEC3CEC4CE450E40E94BC
:101FD000BC2A87FD10C060917305709174058091D3
:101FE0007505909176052DEC3CEC4CE450E40E9494
:101FF000BC2A8823A4F580918F05882331F081E7DE
:1020000096E060E472E00E941D28809104059091A2
:102010000505A0910605B091070520913A0530917C
:102020003B0540913C0550913D05821B930BA40B51
:10203000B50B815A9B4BAD40B04018F08DE290E05B
:1020400063CF85E090E00E94B0050F2EFAE9EF2EF5
:10205000F9E9FF2EF9E90F2FFEE31F2FF02DC8013C
:10206000B70129E23CE54FE05EE30E94572A9B015D
:10207000AC0160918B0570918C0580918D059091DC
:102080008E050E940B2C8823E4F16091420570912B
:10209000430580914405909145052AE037ED43EAD8
:1020A0005CE30E94582A2091C6043091C7044091F5
:1020B000C8045091C9040E94BC2A181614F16091FA
:1020C000B4047091B5048091B6049091B704A8014E
:1020D00097010E94BC2A882321F480911D05882342
:1020E00011F40E94A30DE092B404F092B5040093A1
:1020F000B6041093B70481E080931D0510921C056F
:1021000031C06091C6047091C7048091C804909159
:10211000C9042AE037ED43E25CE30E94572A7B01C1
:102120008C016091B0047091B1048091B2049091DF
:10213000B304A80197010E94BC2A882321F480914E
:102140001C05882311F40E94A30DE092B004F092C4
:10215000B1040093B2041093B30481E080931C0592
:1021600010921D0580911E05882311F40E94E10D37
:102170001F910F91FF90EF9008952F923F924F92F1
:102180005F926F927F928F929F92AF92BF92CF9207
:10219000DF92EF92FF920F931F93DF93CF9300D0C4
:1021A00000D000D0CDB7DEB78091490590914A05A7
:1021B0009E838D8380914D0590914E056D817E812A
:1021C0000E94952CCB014FE652E163E870E40E9437
:1021D00090012091BD053091BE054091BF05509101
:1021E000C0050E94582A69837A838B839C836093FD
:1021F0005705709358058093590590935A0520917F
:1022000010053091110540911205509113052115CB
:1022100031054105510509F448C0609104057091EC
:1022200005058091060590910705621B730B840BD1
:10223000950B0E94592B20E03AEB4BE55AE40E94A3
:10224000C02A29813A814B815C810E940F2C20E0B9
:1022500030E04AE754E40E940F2C2091920530911F
:10226000930540919405509195050E94582A6093DA
:102270009205709393058093940590939505E09053
:10228000DD04F090DE040091DF041091E004A80169
:1022900097010E940B2C181644F4E0929205F092DC
:1022A0009305009394051093950580914F059091A7
:1022B00050056D817E810E94952C882777FD809541
:1022C000982F0E945B2B20E030EC4FE754E40E94F3
:1022D000C02A2FE632E143E850E40E940F2C2AEF97
:1022E00039E146E55FE30E94C02A20E030E040E0AB
:1022F00050E00E94582A1B012C0160935B057093EB
:102300005C0580935D0590935E05809151059091E9
:1023100052056D817E810E94952C882777FD8095DE
:10232000982F0E945B2B20E030EC4FE754E40E9492
:10233000C02A2FE632E143E850E40E940F2C21EE40
:102340003FE641EE5EE30E94C02AA20191010E9495
:10235000572A20E030E040E050E00E94582A3B013C
:102360004C0160935F0570936005809361059093C5
:102370006205C201B101A40193010E94582A7B01A8
:102380008C0180915305909154056D817E810E944E
:10239000952C882777FD8095982F0E945B2B20E055
:1023A00030EC4FE754E40E94C02A2FE632E143E8C4
:1023B00050E40E940F2C2FEF35EE42E95EE30E94BD
:1023C000C02AA80197010E94572A20E030E040E08F
:1023D00050E00E94582A5B016C0160936305709382
:1023E00064058093650590936605C801B701A60151
:1023F00095010E94582A7B018C012091E1043091C3
:10240000E2044091E3045091E4040E94BC2A882332
:1024100044F4E092E104F092E2040093E3041093A8
:10242000E40480915505909156056D817E810E944E
:10243000952C882777FD8095982F0E945B2B20E0B4
:1024400030EC4FE754E40E94C02A2FE632E143E823
:1024500050E40E940F2C27E53FE348E65EE30E942C
:10246000C02A7B018C01CB01D80180936705909332
:102470006805A0936905B0936A0510924E05109205
:102480004D051092500510924F0510925205109272
:102490005105109254051092530510925605109252
:1024A0005505AD81BE81B0934C05A0934B051092AC
:1024B0004A051092490580912C05882309F405C12D
:1024C00080912B05882329F120926B0530926C05B1
:1024D00040926D0550926E0560926F057092700586
:1024E0008092710590927205A0927305B092740566
:1024F000C0927505D09276058E2DD8018093770510
:1025000090937805A0937905B0937A0510922B05E6
:10251000DCC020927B0530927C0540927D05509274
:102520007E0560927F057092800580928105909271
:102530008205A0928305B0928405C0928505D09251
:102540008605C701D8018093870590938805A093DD
:102550008905B0938A0589819A81AB81BC8180937A
:102560008B0590938C05A0938D05B0938E05C201C9
:10257000B101A40193010E940B2C88238CF0C201AD
:10258000B101A60195010E940B2C88234CF02092EA
:10259000420530924305409244055092450521C0C2
:1025A000C401B301A20191010E940B2C88238CF07D
:1025B000C401B301A60195010E940B2C88234CF0A5
:1025C00060924205709243058092440590924505C1
:1025D00008C0A0924205B0924305C0924405D09233
:1025E00045056091C6047091C7048091C80490911C
:1025F000C9042AE037ED43E25DE30E94582A9B01BB
:10260000AC01609142057091430580914405909121
:1026100045050E940B2C1816FCF480912D0588238B
:10262000D9F080911F059091200505979093200582
:1026300080931F0597FF04C01092200510921F057C
:102640000E94A30D80918F05882331F081E796E0E9
:1026500062E572E00E941D2860918B0570918C05E7
:1026600080918D0590918E052091CA043091CB0404
:102670004091CC045091CD040E94572A29E23CE5B8
:102680004FE05EE30E940B2C1816FCF480912D05A0
:102690008823D9F080911F0590912005059790938C
:1026A000200580931F0597FF04C01092200510920B
:1026B0001F050E94A30D80918F05882331F081E7CB
:1026C00096E065E672E00E941D28809104059091D5
:1026D0000505A0910605B09107058093100590931C
:1026E0001105A0931205B093130526960FB6F89422
:1026F000DEBF0FBECDBFCF91DF911F910F91FF9035
:10270000EF90DF90CF90BF90AF909F908F907F9091
:102710006F905F904F903F902F90089580910405A7
:1027200090910505A0910605B091070580932705B6
:1027300090932805A0932905B0932A058091BA04A7
:102740009091BB04A091BC04B091BD04805D974002
:10275000A040B040F1F485E060E070E00E94C12349
:1027600088E060E00E944A2587E061E00E944A25F7
:1027700084E061E00E944A2588EC90E0A0E0B0E0AF
:102780008093BA049093BB04A093BC04B093BD049F
:102790002EC080914605882321F088E061E00E94E8
:1027A0004A2580914705882321F087E060E00E9458
:1027B0004A2580914805882321F084E060E00E944A
:1027C0004A2560911F057091200585E00E94C12374
:1027D00080ED97E0A0E0B0E08093BA049093BB0452
:1027E000A093BC04B093BD0481E080932B0580913D
:1027F000BE049091BF04A091C004B091C104209187
:102800000405309105054091060550910705820F9A
:10281000931FA41FB51F80930C0590930D05A093E3
:102820000E05B0930F05109210051092110510922D
:1028300012051092130508956F927F928F929F92C6
:10284000AF92BF92CF92DF92EF92FF920F931F93BE
:102850008091040590910505A0910605B0910705AA
:1028600080930C0590930D05A0930E05B0930F0572
:102870008EE00E949F2320914D0530914E05280F38
:10288000391F30934E0520934D0500914F0510914F
:1028900050058FE00E949F23080F191F10935005C9
:1028A00000934F05009151051091520580E10E945F
:1028B0009F23080F191F109352050093510581E1C2
:1028C0000E949F237C0180915305909154058E0DA9
:1028D0009F1D909354058093530582E10E949F238E
:1028E0005C0180915505909156058A0D9B1D909332
:1028F0005605809355058091490590914A050196AA
:1029000090934A05809349050027F7FC0095102F06
:10291000C801B7010E945B2B20E030EC4FE754E484
:102920000E94C02A2FE632E143E850E40E940F2CB7
:102930003B014C01CC24B7FCC094DC2CC601B50192
:102940000E945B2B20E030EC4FE754E40E94C02A49
:102950002FE632E143E850E40E940F2C27E53FE3E5
:1029600048E65EE30E94C02A7B018C01C401B301EA
:102970002FEF35EE42E95EE30E94C02A9B01AC01D5
:10298000C801B7010E940B2C181634F48091F10491
:10299000882311F40E9469041F910F91FF90EF901A
:1029A000DF90CF90BF90AF909F908F907F906F906F
:1029B00008958091040590910505A0910605B091B8
:1029C00007058093140590931505A0931605B09301
:1029D000170581E796E062E772E00E942027809168
:1029E000E5049091E6048130910529F481E796E0B1
:1029F00064E772E00EC0009729F481E796E06CE787
:102A000072E007C08F5F9F4F31F481E796E066E880
:102A100072E00E9420276091920570919305809149
:102A20009405909195052091DD043091DE0440914C
:102A3000DF045091E0040E94C02A20E030E048EC1E
:102A400052E40E940F2C0E94282B9B01AC0181E7CD
:102A500096E0B9014AE050E00E94EE2681E796E058
:102A60006FE872E00E94202780912C05882331F0C6
:102A700081E796E061E972E00E94202781E796E015
:102A80006BE972E00E94202780912C05882309F4CD
:102A9000D2C040917B0550917C0560917D0570917D
:102AA0007E0581E796E022E030E00E94072881E77A
:102AB00096E063EA72E00E94202740917F055091E2
:102AC0008005609181057091820581E796E022E0A2
:102AD00030E00E94072881E796E063EA72E00E94F6
:102AE0002027409183055091840560918505709160
:102AF000860581E796E022E030E00E94072881E722
:102B000096E065EA72E00E94202740916B055091A3
:102B10006C0560916D0570916E0581E796E022E08D
:102B200030E00E94072881E796E063EA72E00E94A5
:102B3000202740916F05509170056091710570914B
:102B4000720581E796E022E030E00E94072881E7E5
:102B500096E063EA72E00E9420274091730550914D
:102B60007405609175057091760581E796E022E025
:102B700030E00E94072881E796E06CEA72E00E944C
:102B8000202780914605882329F081E796E061EBB4
:102B900072E004C081E796E063EB72E00E942027B8
:102BA00080914705882329F081E796E061EB72E088
:102BB00004C081E796E063EB72E00E9420278091D9
:102BC0004805882329F081E796E061EB72E004C0B4
:102BD00081E796E063EB72E00E94202780911E055A
:102BE000882331F081E796E065EB72E00E942027B0
:102BF00081E796E067EB72E00E942027409187050D
:102C0000509188056091890570918A0581E796E069
:102C100022E030E00E94072881E796E06DEB72E049
:102C20000E942027409177055091780560917905A1
:102C300070917A0544C040915B0550915C056091AC
:102C40005D0570915E0581E796E022E030E00E942C
:102C5000072881E796E063EA72E00E94202740910E
:102C60005F0550916005609161057091620581E793
:102C700096E022E030E00E94072881E796E063EAD0
:102C800072E00E9420274091630550916405609195
:102C900065057091660581E796E022E030E00E94CC
:102CA000072881E796E063EC72E00E9420274091BC
:102CB0006705509168056091690570916A0581E723
:102CC00096E022E030E00E94072881E796E068EC79
:102CD00072E00E94202760911F057091200581E716
:102CE00096E04AE050E00E94EE2681E796E06EEC26
:102CF00072E00E94202780912C05882349F04091A2
:102D00008B0550918C0560918D0570918E0508C0E2
:102D100040915705509158056091590570915A0599
:102D200081E796E022E030E00E94072881E796E004
:102D300065ED72E00E9420276091920570919305E5
:102D400080919405909195050E94282B9B01AC01E0
:102D500081E796E0B9014AE050E00E94EE2681E763
:102D600096E06BED72E00E9420274091E1045091C3
:102D7000E2046091E3047091E40481E796E022E0CC
:102D800030E00E94072880E090E0A6ECB2E4809357
:102D9000E1049093E204A093E304B093E40481E798
:102DA00096E060EE72E00E9420274091BD055091B0
:102DB000BE056091BF057091C00581E796E022E0F5
:102DC00030E00E94072881E796E065EE72E00E94FD
:102DD00020278091F104882329F081E796E063EBB6
:102DE00072E004C081E796E061EB72E00E94202768
:102DF00081E796E06AEE72E00E94202760919005DC
:102E00007091910581E796E04AE050E00E94EE263D
:102E100081E796E067E671E00E941D280895EF9231
:102E2000FF920F931F93CF93DF93C091CD05D09165
:102E3000CE05C133D105E1F481E796E06FEE72E093
:102E40000E941D2880914605882349F081E796E07D
:102E500060EF72E00E941D2881E090E03DC081E7B4
:102E600096E06BEF72E00E941D2881E090E03EC08A
:102E7000C233D105E1F481E796E06FEE72E00E9483
:102E80001D2880914705882349F081E796E065E099
:102E900073E00E941D2882E090E01EC081E796E06A
:102EA00060E173E00E941D2882E090E01FC0C33300
:102EB000D10501F581E796E06FEE72E00E941D28D2
:102EC00080914805882351F081E796E06AE173E03C
:102ED0000E941D2883E090E060E009C081E796E051
:102EE00065E273E00E941D2883E090E061E00E94AB
:102EF0008E0499C1C033D10529F588E060E00E94B5
:102F00004A2587E061E00E944A2584E061E00E9452
:102F10004A2581E796E06FEE72E00E941D2881E766
:102F200096E06FE273E00E941D2881E796E06FEE65
:102F300072E00E941D2810924605109247051092DB
:102F40004805F6C1C136D105F9F485E060E070E0CE
:102F50000E94C12381E796E06FEE72E00E941D2877
:102F600081E796E06EE373E00E941D2881E796E01A
:102F70006FEE72E00E941D281092200510921F052E
:102F800085E060E070E0A8C1C236D10509F585E0B2
:102F900064E670E00E94C12381E796E06FEE72E084
:102FA0000E941D2881E796E06AE473E00E941D28D4
:102FB00081E796E06FEE72E00E941D2884E690E0C3
:102FC0009093200580931F0585E064E670E084C13E
:102FD000C336D10509F585E068EC70E00E94C12395
:102FE00081E796E06FEE72E00E941D2881E796E08F
:102FF00068E573E00E941D2881E796E06FEE72E0BD
:103000000E941D2888EC90E09093200580931F0576
:1030100085E068EC70E060C1C436D10509F585E053
:103020006FEF70E00E94C12381E796E06FEE72E0DF
:103030000E941D2881E796E066E673E00E941D2845
:1030400081E796E06FEE72E00E941D288FEF90E01E
:103050009093200580931F0585E06FEF70E03CC1E1
:10306000C536D105F9F481E796E06FEE72E00E9473
:103070001D2880911C05882349F010921C0581E7CA
:1030800096E064E773E00E942027CDC081E0809342
:103090001C0581E796E061E873E00E9420270E940A
:1030A000A30DC1C0C636D10569F581E796E06FEE84
:1030B00072E00E941D2880911D05882349F010921E
:1030C0001D0581E796E06DE873E00E9420270BC0A4
:1030D00081E080931D0581E796E069E973E00E9435
:1030E00020270E94A30D81E796E06FEE72E00E9418
:1030F0001D281092100510921105109212051092C1
:10310000130516C1C937D10509F56091B404709152
:10311000B5048091B6049091B7042DEC3CEC4CE4DE
:103120005DE30E94582A6093B4047093B5048093C1
:10313000B6049093B70481E796E06FEE72E00E94C8
:103140001D2881E796E064EA73E06BC0C836D105BC
:1031500009F56091B4047091B5048091B604909122
:10316000B7042DEC3CEC4CE45DE30E94572A6093DD
:10317000B4047093B5048093B6049093B70481E7C8
:1031800096E06FEE72E00E941D2881E796E066EB04
:1031900073E047C0C537D10509F56091B00470915F
:1031A000B1048091B2049091B3042AE037ED43EA70
:1031B0005CE30E94582A6093B0047093B10480933A
:1031C000B2049093B30481E796E06FEE72E00E9440
:1031D0001D2881E796E068EC73E023C0CA36D1056C
:1031E00049F56091B0047091B1048091B20490915E
:1031F000B3042AE037ED43EA5CE30E94572A609368
:10320000B0047093B1048093B2049093B30481E747
:1032100096E06FEE72E00E941D2881E796E06BED6C
:1032200073E00E941D2881E796E06FEE72E00E9435
:103230001D287EC0C936D10531F581E796E06FEED5
:1032400072E00E941D2881E796E060EF73E00E9423
:103250001D2881E796E06FEE72E00E941D288091A4
:103260001F05909120050A969093200580931F05D5
:103270008F3F910561F15CF18FEF90E09093200515
:1032800080931F0524C0CB36D10549F581E796E030
:103290006FEE72E00E941D2881E796E06BEF73E00D
:1032A0000E941D2881E796E06FEE72E00E941D28C3
:1032B00080911F05909120050A9790932005809397
:1032C0001F0597FF04C01092200510921F05609102
:1032D0001F057091200585E00E94C12329C0CF36CB
:1032E000D10531F581E796E06FEE72E00E941D286E
:1032F00081E796E066E074E00E941D2881E796E091
:103300006FEE72E00E941D2880911F0590912005AC
:1033100001969093200580931F058F3F910561F1E1
:103320005CF18FEF90E09093200580931F0524C0FF
:10333000CC36D10549F581E796E06FEE72E00E9448
:103340001D2881E796E060E174E00E941D2881E776
:1033500096E06FEE72E00E941D2880911F0590910B
:10336000200501979093200580931F0597FF04C0C7
:103370001092200510921F0560911F057091200585
:1033800085E00E94C123D2C1C736D10521F581E76E
:1033900096E06FEE72E00E941D2880912D05882333
:1033A00049F081E796E06EE172E00E941D280E94DC
:1033B000A7050CC081E796E064E072E00E941D283A
:1033C00060E070E080E090E00E94C40A81E796E04F
:1033D0006FEE72E0A9C1CA37D10519F40E94E10766
:1033E000A5C1C637D10599F48091DA04882339F054
:1033F0001092DA0481E796E06AE174E095C181E019
:103400008093DA0481E796E067E274E08DC1C83703
:10341000D10529F481E796E063E374E085C1C13703
:10342000D10559F480918F05882319F010928F05EA
:103430007DC181E080938F0579C1C237D10519F430
:103440000E94730773C1C437D10519F40E947F0429
:103450006DC1CD36D10519F40E94690467C1CE361D
:10346000D10519F40E94580461C1C037D10519F47F
:103470000E941D095BC1C737D105A9F480910405DD
:1034800090910505A0910605B0910705805A9541D8
:10349000AF4FBF4F8093A0059093A105A093A205C5
:1034A000B093A30543C1C337D10509F44AC0C4335F
:1034B000D105F1F480E090E00E94B00508E010E052
:1034C00008C08FED95E0B80140E00E9490230F5FA7
:1034D0001F4F8091DB049091DC04019680179107C7
:1034E00084F788E090E09093DC048093DB0429C0AB
:1034F000C234D10519F40E94B10623C0C334D105EA
:1035000019F5809190059091910501978797C8F4DE
:103510008091DB049091DC04089799F080E090E0C2
:103520000E94B0056091DB047091DC046250704031
:103530007093DC046093DB048FED95E040E00E9423
:1035400090230E942405F2C0C533D105E9F480918F
:10355000D1056091CF050E943F28A0E0B0E0BC01FA
:10356000CD010E94592B6093DD047093DE0480939B
:10357000DF049093E0040E94282BDC01CB0162E081
:1035800070E00E94D30203C0C633D10579F481E70D
:1035900096E065E474E00E9420274091DD0450919C
:1035A000DE046091DF047091E004B4C0C733D1053C
:1035B00019F40E94CC02BAC0C833D10599F400E0D6
:1035C00010E08FED95E0B80140E00E9490230F5F7E
:1035D0001F4F82E000301807A1F781E796E064E50D
:1035E00074E0A2C0C933D105E9F46091CF058091A0
:1035F000DD059091DE05039719F080E090E004C0AE
:103600008091D1059091D2050E943F288C010E94A3
:10361000B0050430110509F089C081E796E068EC37
:1036200071E082C0C134D10529F560919205709195
:10363000930580919405909195050E94282BDC01BB
:10364000CB0160E070E00E94D3028091040590916C
:103650000505A0910605B091070580939605909306
:103660009705A0939805B093990581E796E064E6E5
:1036700074E05AC0C434D105E1F58091D105609160
:10368000CF050E943F28EC01BE01882777FD809579
:10369000982F0E945B2B20E030E04AE754E40E9420
:1036A000C02A7B018C0124E333E347E451E40E9408
:1036B0000B2C1816DCF5E092E704F092E804009376
:1036C000E9041093EA04C801B7012AE939E949E19C
:1036D0005FE30E94572A6093AD057093AE05809317
:1036E000AF059093B005CE0166E070E00E94D30272
:1036F00003C0C534D105D1F481E796E068E774E0F2
:103700000E9420274091E7045091E8046091E90469
:103710007091EA0481E796E022E030E00E940728F9
:1037200081E796E067E671E00E941D28DF91CF9166
:103730001F910F91FF90EF900895DF93CF9300D0EA
:10374000CDB7DEB78091040590910505A0910605DF
:10375000B09107058093080590930905A0930A0589
:10376000B0930B0580912C05882309F071C081E787
:1037700096E06EE572E00E94C82540915705509191
:1037800058056091590570915A0581E796E022E04D
:1037900030E00E940A2881E796E064E572E00E942A
:1037A000C82540915B0550915C0560915D05709165
:1037B0005E0581E796E022E030E00E940A2881E77A
:1037C00096E06AE472E00E94C82540915F0550913E
:1037D0006005609161057091620581E796E022E0E5
:1037E00030E00E940A2881E796E060E472E00E94DF
:1037F000C8254091630550916405609165057091FD
:10380000660581E796E022E030E00E940A2881E721
:1038100096E062E372E00E94C82560915B057091BA
:103820005C0580915D0590915E0520915F0530916A
:10383000600540916105509162050E94582A2091CF
:103840006305309164054091650550916605D6C0C9
:1038500081E796E06AE172E00E94C82540918B05FD
:1038600050918C0560918D0570918E0581E796E0F1
:1038700022E030E00E940A2881E796E067E072E0EB
:103880000E94C82540917B0550917C0560917D0583
:1038900070917E0581E796E022E030E00E940A28E0
:1038A00081E796E064EF71E00E94C82540917F05B2
:1038B00050918005609181057091820581E796E0C5
:1038C00022E030E00E940A2881E796E061EE71E094
:1038D0000E94C8254091830550918405609185051B
:1038E0007091860581E796E022E030E00E940A2888
:1038F00081E796E06AEC71E00E94C82560917B0543
:1039000070917C0580917D0590917E0520917F05C9
:103910003091800540918105509182050E94582A7E
:10392000209183053091840540918505509186054D
:103930000E94582AAB01BC0181E796E022E030E00A
:103940000E940A2881E796E06BEB71E00E94C8258F
:1039500040916B0550916C0560916D0570916E05FD
:1039600081E796E022E030E00E940A2881E796E0B5
:103970006CEA71E00E94C82540916F055091700576
:10398000609171057091720581E796E022E030E068
:103990000E940A2881E796E06DE971E00E94C8253F
:1039A000409173055091740560917505709176058D
:1039B00081E796E022E030E00E940A2881E796E065
:1039C0006AE871E00E94C82560916B0570916C05F2
:1039D00080916D0590916E0520916F053091700575
:1039E00040917105509172050E94582A20917305EB
:1039F0003091740540917505509176050E94582AC2
:103A0000AB01BC0181E796E022E030E00E940A2889
:103A100081E796E061E871E00E94C82560911F058A
:103A20007091200581E796E04AE050E00E9401276E
:103A300081E796E062E771E00E94C8254091B004FA
:103A40005091B1046091B2047091B30481E796E0A3
:103A500022E030E00E940A2881E796E064E671E007
:103A60000E94C8254091B4045091B5046091B604F9
:103A70007091B70481E796E022E030E00E940A28C6
:103A800080914605882311F490E007C081E796E015
:103A900065E571E00E94C82591E080914705882383
:103AA00039F081E796E066E471E00E94C82591E074
:103AB00080914805882339F081E796E067E371E05B
:103AC0000E94C82591E080911C05882339F081E788
:103AD00096E06AE271E00E94C82591E080911D05A0
:103AE000882339F081E796E06EE171E00E94C825F5
:103AF00091E080911E05882339F081E796E063E12B
:103B000071E00E94C82502C0992331F081E796E058
:103B10006FEE72E00E941D2881E796E061E171E09E
:103B20000E94C82540910405509105056091060545
:103B30007091070581E796E02AE030E00E949F2619
:103B400081E796E06FE071E00E94C82580912C0526
:103B5000882309F445C040918B0550918C056091F4
:103B60008D0570918E0581E796E022E030E00E949D
:103B7000072881E796E06DE071E00E94C82540913A
:103B80007B0550917C0560917D0570917E0581E7F4
:103B900096E022E030E00E94072881E796E06BE0A3
:103BA00071E00E94C82540917F0550918005609189
:103BB00081057091820581E796E022E030E00E9465
:103BC000072881E796E069E071E00E94C8254091EE
:103BD000830550918405609185057091860544C0E8
:103BE00040915705509158056091590570915A05BB
:103BF00081E796E022E030E00E94072881E796E026
:103C000067E071E00E94C82540915B0550915C051A
:103C100060915D0570915E0581E796E022E030E0FD
:103C20000E94072881E796E065E071E00E94C825C0
:103C300040915F055091600560916105709162054A
:103C400081E796E022E030E00E94072881E796E0D5
:103C500063E071E00E94C8254091630550916405BE
:103C6000609165057091660581E796E022E030E09D
:103C70000E94072881E796E061E071E00E94C82574
:103C800040916705509168056091690570916A05DA
:103C900081E796E022E030E00E94072881E796E085
:103CA0006FEF70E00E94C82560911F05709120059C
:103CB00081E796E04AE050E00E94EE2681E796E038
:103CC0006DEF70E00E940B2681E796E06FEE70E0EA
:103CD0000E94C82560914B0570914C0581E796E0E4
:103CE0004AE050E00E94012781E796E06CED70E029
:103CF0000E94C8254091BD055091BE056091BF0549
:103D00007091C00581E796E022E030E00E940A2829
:103D10008091F104882329F081E796E06CEC70E053
:103D200004C081E796E06DEB70E00E940B26809165
:103D30002C05882319F181E796E06CEA70E00E9477
:103D4000C82540917705509178056091790570916B
:103D50007A0581E796E022E030E00E940A2881E7B8
:103D600096E067E970E00E94C82540918705509170
:103D700088056091890570918A050EC081E796E0FB
:103D80006BE870E00E94C825409167055091680576
:103D90006091690570916A0581E796E022E030E064
:103DA0000E940A288091900590919105892B81F0BD
:103DB00081E796E063E870E00E94C8256091900575
:103DC0007091910581E796E04AE050E00E9401275A
:103DD00081E796E068E770E00E94C825809193062D
:103DE00090919406009711F487E996E0BE016F5F09
:103DF0007F4F681B790B81E796E04AE050E00E9414
:103E0000012781E796E06FEE72E00E941D280F9077
:103E10000F90CF91DF91089581E796E00E94882965
:103E20004091DD055091DE05FA01EE0FFF1FE353CF
:103E3000FA4F91838083BA016F5F7F4F7093DE05E5
:103E40006093DD058D30910519F08A30910591F46C
:103E50002091CD053091CE052533310559F024341C
:103E6000310541F0161617062CF45093DE054093E9
:103E7000DD050DC02091CD053091CE0525333105EE
:103E800019F02434310531F46330710519F40E94BE
:103E90000F1708C08D30910511F00A9739F4613081
:103EA000710521F41092DE051092DD058091040564
:103EB00090910505A0910605B09107058093B50581
:103EC0009093B605A093B705B093B805809190057F
:103ED00090919105479709F040C080E090E00E94E2
:103EE000B0058DEC9CECA4E8B0E48093C6049093FC
:103EF000C704A093C804B093C90483E393E3A3E881
:103F0000B0E48093360590933705A0933805B093BD
:103F1000390583E393E3A3E7B0E48093D604909359
:103F2000D704A093D804B093D9048DEC9CECACE4F6
:103F3000B0E48093ED049093EE04A093EF04B0936B
:103F4000F00480E090E0A0E8BFE38093CA0490937F
:103F5000CB04A093CC04B093CD040895AF92BF924C
:103F6000CF92DF92EF92FF920F931F930E946924EA
:103F70000E94592B20E030E040E85CE30E940F2CC7
:103F80000E942D2B5B016C01809104059091050529
:103F9000A0910605B0910705A816B906CA06DB066A
:103FA00040F4A0922305B0922405C0922505D0923A
:103FB0002605A0920405B0920505C0920605D09290
:103FC0000705809146058823D9F480914705882309
:103FD000B9F480914805882399F480911F05909148
:103FE00020051816190664F080911C05882341F4F9
:103FF00080911D05882321F480912D05882321F0CF
:1040000081E080932C0502C010922C05E090BA0448
:10401000F090BB040091BC041091BD04A601950171
:104020002E193F09400B510B8091270590912805CF
:10403000A0912905B0912A0582179307A407B50717
:1040400058F4AE14BF04C006D10630F080912C05A0
:10405000882311F00E948E13E0900405F09005056E
:104060000091060510910705A80197012A5F3040CD
:10407000404050408091100590911105A09112058B
:10408000B091130582179307A407B50708F52AEF27
:10409000E216F10401051105D8F0809149059091CF
:1040A0004A0518161906A4F40E94BD100E94FE0AC3
:1040B0000E94EF020E9441090E94F1080E94B40888
:1040C0000E9444070E9416070E94E5060E9492077C
:1040D000E0900405F0900505009106051091070594
:1040E000A8019701205D374040405040809108056D
:1040F00090910905A0910A05B0910B0582179307CD
:10410000A407B507E0F480EDE81687E0F80680E044
:10411000080780E0180798F08091BA049091BB04DA
:10412000A091BC04B091BD04883C9105A105B105E6
:1041300031F080918F05882311F00E949D1BE09043
:104140000405F09005050091060510910705A801EA
:1041500097012A5F3040404050408091180590916F
:104160001905A0911A05B0911B0582179307A407A2
:10417000B50780F42AEFE216F1040105110550F0AD
:1041800080911C05882321F480911D05882311F05E
:104190000E94130CE0900405F090050500910605BF
:1041A00010910705A8019701245C39404040504018
:1041B00080912E0590912F05A0913005B091310589
:1041C00082179307A407B50778F484ECE81689E012
:1041D000F80680E0080780E0180730F080912D0590
:1041E000882311F00E940B0FE0900405F090050564
:1041F0000091060510910705A80197012858334141
:10420000404050408091140590911505A0911605ED
:10421000B091170582179307A407B507E0F428E8C3
:10422000E21623E1F20620E0020720E0120798F0F0
:104230008091BA049091BB04A091BC04B091BD04DC
:10424000883C9105A105B10531F080918F05882347
:1042500011F40E94D914E0900405F0900505009136
:10426000060510910705A8019701205E33494440D7
:1042700050408091960590919705A0919805B09136
:10428000990582179307A407B50708F580EEE8168D
:1042900083E9F80684E0080780E01807C0F0E092A0
:1042A0009605F092970500939805109399056091F3
:1042B00092057091930580919405909195050E94C7
:1042C000282BDC01CB0160E070E00E94D30220913A
:1042D000C1053091C2054091C3055091C40580913C
:1042E000040590910505A0910605B09107052817D2
:1042F00039074A075B0738F4211531054105510597
:1043000011F00E94E1078091CB059091CC050E94AD
:104310004603E0900405F090050500910605109114
:104320000705A801970120583F4442415040809121
:10433000B5059091B605A091B705B091B805821763
:104340009307A407B507A8F420E8E2162FE4F206C5
:1043500022E1020720E0120760F0E092B505F0923A
:10436000B6050093B7051093B80587E190E00E9469
:10437000B0058091040590910505A0910605B091C6
:104380000705209123053091240540912505509182
:104390002605821B930BA40BB50B815C944DA140A9
:1043A000B04040F080911E05882321F08CE290E01F
:1043B0000E94B005A0900405B0900505C0900605C8
:1043C000D0900705E090AC04F090AD040091AE04ED
:1043D0001091AF04A60195012E193F09400B510B16
:1043E00080910C0590910D05A0910E05B0910F05DF
:1043F00082179307A407B50738F4AE14BF04C006AC
:10440000D10610F00E941C1481E796E00E94572903
:10441000181619067CF48091BA049091BB04A091FF
:10442000BC04B091BD04883C9105A105B10511F013
:104430000E940C1F2091A0053091A1054091A2057A
:104440005091A305211531054105510579F1809160
:10445000040590910505A0910605B0910705821706
:104460009307A407B50710F1609192057091930529
:1044700080919405909195050E94282BDC01CB0139
:1044800060E070E00E94D3020E94C9040E9473079A
:1044900081E796E067E874E00E941D281092A0056D
:1044A0001092A1051092A2051092A3051F910F91E1
:1044B000FF90EF90DF90CF90BF90AF900895AF92B4
:1044C000BF92CF92DF92EF92FF920F931F9380E003
:1044D0000E949C238EE060E00E940B258FE060E04C
:1044E0000E940B2580E160E00E940B2581E160E0E5
:1044F0000E940B2582E160E00E940B2588E061E0CC
:104500000E940B2587E061E00E940B2584E061E0BA
:104510000E940B2588E060E00E944A2587E061E068
:104520000E944A2584E061E00E944A2585B5887F83
:10453000816085BD8DE061E00E940B258DE060917A
:10454000CB050E944A2585E061E00E940B25609121
:104550001F057091200585E00E94C12383E061E082
:104560000E940B2583E061E00E944A2582E061E021
:104570000E940B2582E060E00E944A2581E796E0D8
:1045800040E052EC61E070E00E94D02881E796E0C4
:1045900066E974E00E941D2882E090E00E94060512
:1045A0009C01181619067CF4B901882777FD8095BF
:1045B000982F0E945B2B6093DD047093DE04809340
:1045C000DF049093E00480E090E00E940605AA27B3
:1045D00097FDA095BA2FBC01CD010E945B2B5B011A
:1045E0006C01E090DD04F090DE040091DF04109196
:1045F000E004A80197010E940B2C18164CF4E092DD
:104600009205F0929305009394051093950508C0C8
:10461000A0929205B0929305C0929405D092950510
:1046200084E090E00E9406059C010097B9F0285EA6
:104630003340B901882777FD8095982F0E945B2B26
:1046400020E030E04AE754E40E94C02A6093BD05B0
:104650007093BE058093BF059093C00586E090E0FF
:104660000E940605AA2797FDA095BA2FBC01CD018F
:104670000E945B2B20E030E04AE754E40E94C02A0D
:104680007B018C0124E333E347E451E40E940B2CCB
:1046900018167CF5E092E704F092E8040093E90430
:1046A0001093EA04C801B7012AE939E949E15FE357
:1046B0000E94572A6093AD057093AE058093AF05B5
:1046C0009093B00516C00E9406050097C9F090931C
:1046D0009105809390058731910511F00E94B005F6
:1046E0008091DB049091DC0402969093DC0480932B
:1046F000DB048091DB049091DC04813291051CF392
:104700001F910F91FF90EF90DF90CF90BF90AF90EF
:104710000895F999FECF72BD61BDF89A80B50895EC
:10472000F999FECF1FBA72BD61BD40BD0FB6F894B6
:10473000FA9AF99A0FBE08958093F2040895982F7B
:104740008E3008F09E5097708091F2048295880F09
:10475000880F807C892B80937C0080917A00806414
:1047600080937A0080917A0086FDFCCF20917800BA
:1047700040917900942F80E030E0282B392BC9013B
:1047800008951F93CF93DF93182FEB0161E00E94F0
:104790000B25209709F44AC0CF3FD10509F449C041
:1047A000E12FF0E0ED54FD4F84918330C1F084306F
:1047B00028F4813051F08230B1F50CC0863019F107
:1047C000873049F1843079F514C084B5806884BDA0
:1047D000C7BD33C084B5806284BDC8BD2EC0809182
:1047E0008000806880938000D0938900C093880007
:1047F00024C080918000806280938000D0938B00E1
:10480000C0938A001AC08091B00080688093B00085
:10481000C093B30012C08091B00080628093B0005A
:10482000C093B4000AC0C038D1051CF4812F60E0E9
:1048300002C0812F61E00E944A25DF91CF911F9134
:1048400008951F920F920FB60F9211242F933F934A
:104850008F939F93AF93BF938091E4059091E5056B
:10486000A091E605B091E7053091E8050196A11DFC
:10487000B11D232F2D5F2D3720F02D570196A11D3F
:10488000B11D2093E8058093E4059093E505A0937E
:10489000E605B093E7058091E0059091E105A091D0
:1048A000E205B091E3050196A11DB11D8093E005DD
:1048B0009093E105A093E205B093E305BF91AF911A
:1048C0009F918F913F912F910F900FBE0F901F904E
:1048D00018958FB7F8942091E4053091E505409143
:1048E000E6055091E7058FBFB901CA0108959B0104
:1048F000AC017FB7F8948091E0059091E105A0911B
:10490000E205B091E30566B5A89B05C06F3F19F0BD
:104910000196A11DB11D7FBFBA2FA92F982F8827FF
:10492000860F911DA11DB11D62E0880F991FAA1F5E
:10493000BB1F6A95D1F7BC012DC0FFB7F8948091D9
:10494000E0059091E105A091E205B091E305E6B59F
:10495000A89B05C0EF3F19F00196A11DB11DFFBF37
:10496000BA2FA92F982F88278E0F911DA11DB11D39
:10497000E2E0880F991FAA1FBB1FEA95D1F7861B9B
:10498000970B885E9340C8F2215030404040504021
:1049900068517C4F211531054105510571F6089587
:1049A000789484B5826084BD84B5816084BD85B50A
:1049B000826085BD85B5816085BDEEE6F0E08081D1
:1049C00081608083E1E8F0E01082808182608083F2
:1049D000808181608083E0E8F0E080818160808375
:1049E000E1EBF0E0808184608083E0EBF0E08081A7
:1049F00081608083EAE7F0E0808184608083808149
:104A000082608083808181608083808180688083F0
:104A10001092C1000895CF93DF93482F50E0CA0150
:104A200081569D4FFC01349145575D4FFA018491A9
:104A3000882369F190E0880F991FFC01E359FD4F2D
:104A4000A591B491FC01E958FD4FC591D49166231D
:104A500051F42FB7F8948C91932F909589238C93D0
:104A6000888189230BC0623061F42FB7F8948C9150
:104A7000932F909589238C938881832B88832FBFD4
:104A800006C09FB7F8948C91832B8C939FBFDF91C6
:104A9000CF910895482F50E0CA018D549D4FFC01DD
:104AA0002491CA0181569D4FFC01949145575D4F59
:104AB000FA013491332309F440C0222351F1233009
:104AC00071F0243028F42130A1F0223011F514C007
:104AD0002630B1F02730C1F02430D9F404C08091E1
:104AE00080008F7703C0809180008F7D809380004D
:104AF00010C084B58F7702C084B58F7D84BD09C096
:104B00008091B0008F7703C08091B0008F7D80933B
:104B1000B000E32FF0E0EE0FFF1FE958FD4FA59125
:104B2000B4912FB7F894662321F48C919095892342
:104B300002C08C91892B8C932FBF0895CF92DF9266
:104B4000EF92FF920F931F93CF93DF937C016B0142
:104B50008A01C0E0D0E00FC0D6016D916D01D70190
:104B6000ED91FC910190F081E02DC7010995C80FEE
:104B7000D91F015010400115110571F7CE01DF91C9
:104B8000CF911F910F91FF90EF90DF90CF900895FC
:104B9000EF92FF920F931F93CF93DF937C018B01D2
:104BA000C0E0D0E0F8010F5F1F4F6491662359F019
:104BB000D701ED91FC910190F081E02DC70109959D
:104BC000C80FD91FEFCFCE01DF91CF911F910F9169
:104BD000FF90EF900895EF92FF920F931F938C0137
:104BE000DC01ED91FC910190F081E02D6DE00995E3
:104BF0007C01D801ED91FC910190F081E02DC8017C
:104C00006AE009959C012E0D3F1DC9011F910F916E
:104C1000FF90EF900895EF92FF920F931F937C0106
:104C20000E94C8258C01C7010E94EB259C01200F22
:104C3000311FC9011F910F91FF90EF900895CF93FD
:104C4000DF93EC016115710519F420E030E00FC02D
:104C5000DB010D900020E9F71197A61BB70BE88147
:104C6000F9810280F381E02DAD0109959C01C90114
:104C7000DF91CF9108954F925F927F928F929F9292
:104C8000AF92BF92CF92DF92EF92FF920F931F935A
:104C9000DF93CF93CDB7DEB7A1970FB6F894DEBF01
:104CA0000FBECDBF2C01742ECB01223008F42AE0B8
:104CB00019A231E2C32ED12CCC0EDD1E822E9924F6
:104CC000AA24BB24672D752FA50194010E94A82C4E
:104CD00079018A01C801B701A50194010E94762CCF
:104CE000472D461B0894C108D1084A3014F4405D92
:104CF00001C0495CF6014083E114F104010511058E
:104D000021F07E2C5F2DC801DDCFC201B6010E94CB
:104D10001F26A1960FB6F894DEBF0FBECDBFCF9170
:104D2000DF911F910F91FF90EF90DF90CF90BF9098
:104D3000AF909F908F907F905F904F900895DC018F
:104D40002115310541F4ED91FC910190F081E02DA8
:104D5000642F099508950E943B260895CF92DF9213
:104D6000EF92FF920F931F93CF93DF93EC016A01B1
:104D70007B012115310541F4E881F9810190F08131
:104D8000E02D642F09951FC02A303105D1F477FF3B
:104D900017C0E881F9810190F081E02D6DE209955D
:104DA0008C0144275527BA014C195D096E097F090A
:104DB000CE012AE00E943B269801280F391F04C02B
:104DC0002AE00E943B269C01C901DF91CF911F91EF
:104DD0000F91FF90EF90DF90CF900895EF92FF92A8
:104DE0000F931F937B019A010027F7FC0095102F6A
:104DF000B801A7010E94AE261F910F91FF90EF907E
:104E00000895CF92DF92EF92FF920F931F936C0160
:104E10007B019A010027F7FC0095102FB801A7012C
:104E20000E94AE268C01C6010E94EB25080F191FB7
:104E3000C8011F910F91FF90EF90DF90CF900895E0
:104E40000E941F2608957F928F929F92AF92BF92E9
:104E5000CF92DF92EF92FF920F931F93CF93DF9346
:104E60004C017A018B01722ECB01BA01A801970186
:104E70000E94722C882321F0C4016EE974E021C0E5
:104E8000C0E0D0E057016801E894D7F8C601B50149
:104E90002FEF3FEF4FE75FE70E94722C882351F41A
:104EA000C601B5012FEF3FEF4FE75FE70E94BC2A35
:104EB000181614F0C1E0D0E0219739F0C40162EA7D
:104EC00074E00E941F26EC0193C0C801B7012FEFC8
:104ED0003FEF4FE75FE40E940B2C181654F0C80117
:104EE000B7012FEF3FEF4FE75FEC0E94BC2A88230A
:104EF00024F4C40166EA74E0E4CFC801B70120E0FD
:104F000030E040E050E00E94BC2A87FD03C0C0E0D2
:104F1000D0E00EC0D401ED91FC910190F081E02D24
:104F2000C4016DE20995EC0117FB109517F9109576
:104F300020E030E040E05FE3DD240BC0CA01B901AE
:104F400020E030E040E251E40E94C02A9B01AC0125
:104F5000D394D71498F3C801B7010E94582A5B0173
:104F60006C010E942D2B7B018C01C401B801A701AB
:104F70002AE030E00E949F26C80FD91F772039F021
:104F8000C4016AEA74E00E941F26C80FD91FC80135
:104F9000B7010E94592B9B01AC01C601B5010E94CB
:104FA000572A24C020E030E040E251E40E940F2C58
:104FB0007B018C010E94282B5B016C01CC24B7FC87
:104FC000C094DC2CC401B601A5012AE030E00E94A7
:104FD000AE26C80FD91FC601B5010E945B2B9B01ED
:104FE000AC01C801B7010E94572A7A947720D1F604
:104FF000CE01DF91CF911F910F91FF90EF90DF9045
:10500000CF90BF90AF909F908F907F9008950E9417
:1050100023270895EF92FF920F931F937C010E9424
:1050200023278C01C7010E94EB25080F191FC80117
:105030001F910F91FF90EF900895EF92FF920F93C1
:105040001F937C010E941F268C01C7010E94EB2543
:10505000080F191FC8011F910F91FF90EF9008953D
:10506000CF93DF930E94D0240E945F22C2E8D8E24F
:105070000E94AE1F2097E1F30E948228F9CF70E0D2
:10508000382F20E0622B732BCB01089508951F92D7
:105090000F920FB60F9211242F933F934F938F933C
:1050A0009F93EF93FF938091C00082FD1DC04091BC
:1050B000C6002091290630912A062F5F3F4F2F739B
:1050C000307080912B0690912C062817390771F0CB
:1050D000E0912906F0912A06E751FA4F4083309378
:1050E0002A062093290602C08091C600FF91EF9105
:1050F0009F918F914F913F912F910F900FBE0F90E5
:105100001F901895E0917D06F0917E06E05CFF4FC0
:105110008191919120813181821B930B8F739070CB
:10512000892B11F00E94462808951F920F920FB606
:105130000F9211242F933F938F939F93EF93FF939D
:1051400020916D0630916E0680916F0690917006E9
:105150002817390731F48091C1008F7D8093C100F9
:1051600014C0E0916F06F0917006E35DF94F208165
:1051700080916F069091700601968F739070909356
:10518000700680936F062093C600FF91EF919F9168
:105190008F913F912F910F900FBE0F901F901895F8
:1051A000AF92BF92DF92EF92FF920F931F93CF9334
:1051B000DF93EC017A018B01DD24403081EE58074A
:1051C00080E0680780E0780711F0DD24D39491E057
:1051D000A92EB12CEC89FD89DD2069F0C50108A05C
:1051E00002C0880F991F0A94E2F7808360E079E09B
:1051F0008DE390E005C0108260E874E88EE190E0F5
:10520000A80197010E94A82C2150304040405040F6
:10521000569547953795279580E12030380720F03F
:10522000DD2011F0DD24D6CFE889F9893083EA89C1
:10523000FB89208319A2EE89FF89408121E030E0BB
:10524000C9010C8C02C0880F991F0A94E2F7482B01
:105250004083EE89FF894081C9010D8C02C0880F0F
:10526000991F0A94E2F7482B4083EE89FF89408119
:10527000C9010E8C02C0880F991F0A94E2F7482BCF
:105280004083EE89FF8980810F8C02C0220F331F7B
:105290000A94E2F7209528232083DF91CF911F9174
:1052A0000F91FF90EF90DF90BF90AF900895DC01D9
:1052B0001C96ED91FC911D97E05CFF4F219131917F
:1052C00080819181281B390B2F733070C90108959B
:1052D000DC011C96ED91FC911D97E05CFF4F208155
:1052E0003181E054F040DF01AE5BBF4F8D919C9166
:1052F00011972817390719F42FEF3FEF07C08D9149
:105300009C91E80FF91F8081282F30E0C901089592
:10531000DC011C96ED91FC911D97E05CFF4F208114
:105320003181E054F040DF01AE5BBF4F8D919C9125
:1053300011972817390719F42FEF3FEF10C08D91FF
:105340009C911197E80FF91F20818D919C911197E5
:1053500001968F73907011969C938E9330E0C901E3
:105360000895DC0191968C919197882339F0549699
:10537000ED91FC915597808186FFF9CF91961C9213
:105380000895CF93DF93EC01EE85FF85E05CFF4F3E
:1053900020813181E054F0402F5F3F4F2F733070F8
:1053A000DF01AE5BBF4F8D919C9111972817390794
:1053B000D1F3E05CFF4F80819181E054F040E80F31
:1053C000F91F6083EE85FF85E05CFF4F318320830A
:1053D000EE89FF89208181E090E00F8C02C0880F68
:1053E000991F0A94E2F7282B208381E089A3EC8996
:1053F000FD8980818064808381E090E0DF91CF919E
:105400000895109274061092730688EE93E0A0E05F
:10541000B0E08093750690937606A0937706B093DC
:10542000780687EF94E0909372068093710689EE78
:1054300095E090937E0680937D068DE296E09093B2
:10544000800680937F0685EC90E09093820680939F
:10545000810684EC90E0909384068093830680EC30
:1054600090E0909386068093850681EC90E090937F
:1054700088068093870682EC90E090938A0680935A
:10548000890686EC90E090938C0680938B0684E0EE
:1054900080938D0683E080938E0687E080938F064D
:1054A00085E08093900681E080939106089550589E
:1054B000BB27AA270ED075C166D130F06BD120F082
:1054C00031F49F3F11F41EF45BC10EF4E095E7FB4D
:1054D00051C1E92F77D180F3BA17620773078407A8
:1054E000950718F071F49EF58FC10EF4E0950B2E20
:1054F000BA2FA02D0B01B90190010C01CA01A00126
:105500001124FF27591B99F0593F50F4503E68F180
:105510001A16F040A22F232F342F4427585FF3CFC1
:10552000469537952795A795F0405395C9F77EF492
:105530001F16BA0B620B730B840BBAF09150A1F0DB
:10554000FF0FBB1F661F771F881FC2F70EC0BA0F61
:10555000621F731F841F48F4879577956795B795E9
:10556000F7959E3F08F0B3CF9395880F08F09927E1
:10557000EE0F979587950895D9D008F481E00895A6
:105580000CD00FC107D140F0FED030F021F45F3FC6
:1055900019F0F0C0511139C1F3C014D198F3992317
:1055A000C9F35523B1F3951B550BBB27AA276217E7
:1055B0007307840738F09F5F5F4F220F331F441F2C
:1055C000AA1FA9F333D00E2E3AF0E0E830D0915064
:1055D0005040E695001CCAF729D0FE2F27D0660F51
:1055E000771F881FBB1F261737074807AB07B0E890
:1055F00009F0BB0B802DBF01FF2793585F4F2AF0A6
:105600009E3F510568F0B6C000C15F3FECF3983E85
:10561000DCF3869577956795B795F7959F5FC9F702
:10562000880F911D9695879597F90895E1E0660F8B
:10563000771F881FBB1F621773078407BA0720F004
:10564000621B730B840BBA0BEE1F88F7E09508956D
:1056500004D06894B111D9C00895BCD088F09F5788
:1056600090F0B92F9927B751A0F0D1F0660F771FAE
:10567000881F991F1AF0BA95C9F712C0B13081F08E
:10568000C3D0B1E00895C0C0672F782F8827B85FD6
:1056900039F0B93FCCF3869577956795B395D9F7EF
:1056A0003EF490958095709561957F4F8F4F9F4FF9
:1056B0000895E89409C097FB3EF490958095709505
:1056C00061957F4F8F4F9F4F9923A9F0F92F96E94E
:1056D000BB279395F695879577956795B795F111C3
:1056E000F8CFFAF4BB0F11F460FF1BC06F5F7F4F60
:1056F0008F4F9F4F16C0882311F096E911C0772372
:1057000021F09EE8872F762F05C0662371F096E87A
:10571000862F70E060E02AF09A95660F771F881F49
:10572000DAF7880F9695879597F90895990F0008ED
:10573000550FAA0BE0E8FEEF16161706E807F90763
:10574000C0F012161306E407F50798F0621B730BFE
:10575000840B950B39F40A2661F0232B242B252B7F
:1057600021F408950A2609F4A140A6958FEF811D22
:10577000811D089597F99F6780E870E060E00895C3
:105780009FEF80EC089500240A9416161706180659
:105790000906089500240A94121613061406050635
:1057A0000895092E0394000C11F4882352F0BB0FC6
:1057B00040F4BF2B11F460FF04C06F5F7F4F8F4F29
:1057C0009F4F089557FD9058440F551F59F05F3F64
:1057D00071F04795880F97FB991F61F09F3F79F013
:1057E00087950895121613061406551FF2CF469595
:1057F000F1DF08C0161617061806991FF1CF869517
:105800007105610508940895E894BB2766277727FA
:10581000CB0197F908958ADF08F48FEF08950BD034
:10582000C0CFB1DF28F0B6DF18F0952309F0A2CF82
:10583000A7CF1124EACFC6DFA0F3959FD1F3950F30
:1058400050E0551F629FF001729FBB27F00DB11D04
:10585000639FAA27F00DB11DAA1F649F6627B00D94
:10586000A11D661F829F2227B00DA11D621F739F7D
:10587000B00DA11D621F839FA00D611D221F749F8B
:105880003327A00D611D231F849F600D211D822FD2
:10589000762F6A2F11249F5750408AF0E1F0882319
:1058A0004AF0EE0FFF1FBB1F661F771F881F915026
:1058B0005040A9F79E3F510570F05CCFA6CF5F3FE7
:1058C000ECF3983EDCF3869577956795B795F79559
:1058D000E7959F5FC1F7FE2B880F911D96958795E1
:1058E00097F9089523DF880B990B0895629FD001E3
:1058F000739FF001829FE00DF11D649FE00DF11D8B
:10590000929FF00D839FF00D749FF00D659FF00D39
:105910009927729FB00DE11DF91F639FB00DE11D26
:10592000F91FBD01CF011124089597FB092E072609
:105930000AD077FD04D02ED006D000201AF470953E
:1059400061957F4F0895F6F7909581959F4F089543
:10595000A1E21A2EAA1BBB1BFD010DC0AA1FBB1F73
:10596000EE1FFF1FA217B307E407F50720F0A21BE5
:10597000B30BE40BF50B661F771F881F991F1A9452
:1059800069F760957095809590959B01AC01BD017C
:10599000CF010895AA1BBB1B51E107C0AA1FBB1F63
:1059A000A617B70710F0A61BB70B881F991F5A95AB
:1059B000A9F780959095BC01CD010895EE0FFF1FCA
:0C59C0000590F491E02D0994F894FFCFBD
:1059CC003C77616C6C706F7765723E0062617474C9
:1059DC00506C757350696E20484947482028666C96
:1059EC006F77290062617474506C757350696E2006
:1059FC004C4F5720286E6F20666C6F7729006261C0
:105A0C007474207361666574792073776974636844
:105A1C00204F4E003C706F7765725F6572726F72CB
:105A2C002000303E002C003E0077726974696E676E
:105A3C00206572726F7220746F20656570726F6D65
:105A4C000062617474207361666574792073776980
:105A5C00746368204F4646003C686967685F6375ED
:105A6C007272656E743E000A7A65726F206375728D
:105A7C0072656E740A006E65772063757272656E5E
:105A8C00742063616C3A20003C7265646F636B3EFA
:105A9C00003C73687574646F776E3E0064616E676A
:105AAC0065726F75736C79206C6F772063656C6CA5
:105ABC00003C636861726765643E003C646F636BB5
:105ACC0065643E006175746F206368617267652060
:105ADC004F4E003C756E646F636B65643E00617580
:105AEC00746F20636861726765204F4646000A6DCB
:105AFC006178206368617267652074696D650A005E
:105B0C000A707265636F6E646974696F6E696E6733
:105B1C000A0068696768204348415247494E47204C
:105B2C0063656C6C00686967682063757272656E7A
:105B3C0074003C00646F636B65642000756E646F69
:105B4C00636B65642000756E6B6E6F776E2000253D
:105B5C00005F6368617267696E67002063656C6CD7
:105B6C00733A005F005F69646C653A005F73683A72
:105B7C00003100300041005F7343563A005F7349B7
:105B8C00563A005F73563A005F70776D3A005F616A
:105B9C006D70733A005F6D41683A005F6C563A0065
:105BAC005F63433A005F62503A005F65523A00000F
:105BBC007368756E7431204F4646007368756E7449
:105BCC0031204F4E007368756E7432204F4646007C
:105BDC007368756E7432204F4E007368756E743333
:105BEC00204F4646007368756E7433204F4E007319
:105BFC0068756E747320616C6C206F666600766FCE
:105C0C006C74732050574D203000766F6C74732079
:105C1C0050574D2031303000766F6C7473205057D4
:105C2C004D2032303000766F6C74732050574D20FD
:105C3C003235350061646A566F6C7473204F46467A
:105C4C000061646A566F6C7473204F4E0061646A15
:105C5C00416D7073204F46460061646A416D7073EC
:105C6C00204F4E0074617267657420416D70732013
:105C7C002B302E30350074617267657420416D7065
:105C8C0073202D302E303500746172676574207668
:105C9C006F6C7473202B302E303200746172676518
:105CAC007420766F6C7473202D302E30323A2000B5
:105CBC0070777250574D202B3130007077725057DF
:105CCC004D202D31300070777250574D202B310004
:105CDC0070777250574D202D310066756C6C617564
:105CEC00746F204F46460066756C6C6175746F203E
:105CFC004F4E003C69643A3A6F63756C7573506F24
:105D0C007765723E003C6D416843617061636974F4
:105D1C00793A20003C656570726F6D5F65726173D6
:105D2C0065643E003C77726974696E675F746F5F7F
:105D3C00656570726F6D3E003C646F636B566F6C83
:105D4C00746167653A20003C5348555454494E479A
:105D5C00444F574E3E003C72657365743E006E6155
:105D6C006E00696E66006F7666002E000A000000F9
:105D7C00333383400000003F0500D00700003200A1
:105D8C000000C4090000CDCC84400000803F009787
:105D9C00490160EA00003333734001080000D084ED
:105DAC00450000C642FFFF00006041FFFFCDCC4C18
:105DBC0040010100000000C1299E2557298829684F
:045DCC0029B12900D0
:00000001FF
